:020000040000FA
:06000000FFEF25F01200E5
:020006001200E6
:0600080004EF08F01200F5
:02000E000014DC
:08001000032A2C01010000008D
:060018000CEF08F01200DD
:02001E000200DE
:10002000794C0000910500005D0000000E0000000A
:08003000EE0500000A000000CB
:0800380058EC05F0FB0EDBCFD4
:10004000F3FFDB06F35000090AE0A6EC05F0FA0E18
:1000500011EC06F0F3E1261CF1E1010E01D0000ED7
:1000600087EF05F058EC05F03B0EE12402E3E16870
:10007000E652E16E010EDB6A020EDB6AF90EDBCF9F
:10008000F6FFFA0EDBCFF7FFFB0EDBCFF8FF080021
:10009000F550DF6EDF5002E1ABEF04F0250EDF5CC0
:1000A00002E09EEF04F0030EDB6A040EDB6A050E2D
:1000B000DB6A060EDB6A070EDB6AC0EC04F02D0E6D
:1000C000DF5C0CE02B0EDF5C09E0200EDF5C06E05D
:1000D000230EDF5C03E0300EDF5C1AE1DF50300AF4
:1000E00014E0130A0FE0030A0AE00B0A05E0060A0F
:1000F000E4E1030EDB80E1D7030EDB82DED7030EE3
:10010000DB84DBD7030EDB86D8D7030EDB88D5D79D
:100110002A0EDF5C1BE1BCEC04F00AEC05F010E0F9
:10012000030EDB8006680768130EDBCF0DF0140E9C
:10013000DBCF0EF0D2EC07F0040E04C0DBFF03D0DF
:10014000130EF3EC04F0C0EC04F00BD0090EDB6AE4
:1001500061EC05F003E0D5EC05F0FAD7090EF3ECFD
:1001600004F0030EDBB0DB982E0EDF5C1BE1C0EC6D
:1001700004F02A0EDF5C0BE1BCEC04F00AEC05F0A5
:1001800003E1130E45EC05F0C0EC04F00BD0090EB2
:10019000DB6A61EC05F003E0D5EC05F0FAD7090E57
:1001A00045EC05F0680EDF5C07E1C0EC04F0680E7A
:1001B000DF5C1DE1030E18D0740EDF5C17E07A0ED1
:1001C000DF5C14E0480EDF5C06E0540EDF5C03E009
:1001D0005A0EDF5C02E1020E07D06C0EDF5C03E01A
:1001E0006A0EDF5C04E1010E98EC05F0C9DBDF501C
:1001F0006E0A01E17FD31E0A01E192D1200A01E1DA
:100200008FD13F0A01E149D11A0A01E146D10D0A15
:1002100001E143D1200A01E140D13A0A01E13DD197
:10022000200A01E13AD1260A01E135D10D0A01E1A6
:1002300032D11A0A01E1D9D0200A4AE0300A1FE07F
:10024000460A0EE0250A01E083D3D950F90FE96E82
:10025000FF0EDA20EA6E010EEE5E000EEE5AEE5A46
:10026000A6EC05F0250EE66E95DB03E1261C01E108
:1002700069D3A2EC05F001E26BD3DB2A69D3080E47
:10028000DB6A040EDB50010806E2040EDB046AECB4
:1002900005F0DB508BDB080EDB5009E0030EDB5072
:1002A000010B05E172DB01E04DD3080EDB6A64DB74
:1002B000EFCFDFFF1AEC06F003E1261C01E142D389
:1002C000A2EC05F001E3DB2A60DB01E141D33AD384
:1002D000070EDB5002080FE1E6EC05F0030EADEC73
:1002E00005F00E0EEECFDBFF0F0EEECFDBFF100E94
:1002F000EECFDBFF20D0F70EDBCF28F0F80EDBCF00
:1003000029F0020E285E000E295AF70E28C0DBFFE6
:10031000F80E29C0DBFF28C0E9FF29C0EAFF9DECE9
:1003200005F0276A0E0E25C0DBFF0F0E26C0DBFF8F
:10033000100E27C0DBFF0E0EDBCFE6FF0F0EDBCF6C
:10034000E6FF100EDBCFE6FF62EC23F0E552E5524C
:10035000E552130E05C0DBFF140E06C0DBFF060ED0
:10036000DB5005E0130EE1EC05F001E26ADB05EC81
:1003700006F002E2130E37DBC8EC05F006E0040ECF
:10038000E1EC05F002E2050E2EDB030EDBB005D03A
:10039000FCDA01E0D7D2080EDB6A090EDB6A0E0E2A
:1003A000DBCFF6FF0F0EDBCFF7FF100EDBCFF8FF32
:1003B0000800F550DF6EDF5014E00BEC06F011E2A0
:1003C0001AEC06F003E1261C01E1BCD2BBDB01E321
:1003D000DB2A090EDB2AD9500E0FE96E000ECBDBAB
:1003E000E7D7D3DA01E1B4D2ADD2C6DA110EEECF3F
:1003F000DBFF120EEDCFDBFF110EDBCFE6FF120E9F
:10040000DBCFE6FFA8EC23F0E552E552130EF3CF65
:10041000DBFF140EF4CFDBFF060EDB5004E0130EFF
:10042000D0DB01E20EDB05EC06F002E2130EDBDAB4
:10043000AFDB05E0040EC5DB02E2050ED4DA030EE5
:10044000DBB005D0A2DA01E07DD2080EDB6A090E2E
:10045000DB6A110EDBCFE9FF120EDBCFEAFFEFCF35
:10046000DFFFDF5014E0D7DB12E2E4DB03E1261C00
:1004700001E168D267DB01E3DB2A090EDB2A110EFA
:10048000DB2ADBCFE9FF120EE8E3DB2AE6D77DDAD1
:1004900001E15ED257D2030EDB8E070EDB0410E1C2
:1004A00095DB040E5ADB0A0EEECFDBFF0B0EEECF10
:1004B000DBFF0C0EEECFDBFF0D0EEECFDBFF6CD0C3
:1004C000070EDB5003082CE1030EDBAE0DD0B2DAD1
:1004D000020E76DAEFCF25F0266A276A286A25AE63
:1004E00039D02668276835D0F70EDBCF26F0F80E16
:1004F000DBCF27F0020E265E000E275AF70E26C02D
:10050000DBFFF80E27C0DBFF26C0E9FF27C0EAFFAC
:10051000EFCF25F00A0E25C0DBFF0B0EDB6A38D0CB
:10052000070EDB50020809E1030EDBAE04D059DBF5
:1005300027AE10D00ED055DB0DD0030EDBAE12D09F
:1005400079DA020E3DDAF9DA276A286A26AE02D095
:1005500027682868E2DA0C0E27C0DBFF0D0E28C0E2
:10056000DBFF1AD0F70EDBCF27F0F80EDBCF28F039
:10057000020E275E000E285AF70E27C0DBFFF80E8A
:1005800028C0DBFF27C0E9FF28C0EAFFD6DAC5DABA
:100590000C0EDB6A0D0EDB6A060EDB5005E1010E68
:1005A000F36E050EF3CFDBFF150EDB6A160EDB6A6A
:1005B000D950370F256E000EDA20266E390E25C071
:1005C000DBFF3A0E26C0DBFF380EDB6A080EDB6A63
:1005D0000A0EAEDADF50780A12E0200A10E0280A8C
:1005E0000CE0200A0AE03F0A06E00D0A02E0200AB9
:1005F00008E1020E05D0080E03D0080EDF26100E0B
:1006000097DA030EDBBE02D0DB92DB94DB50800B6B
:1006100024E08ADAD890030EEB50000A08E6000EB8
:10062000EE5C000EEE58000EEE58000EEE5815E28D
:1006300013DA0B680C680D680E6869EC25F00A0E79
:1006400000C0DBFF0B0E01C0DBFF0C0E02C0DBFFA6
:100650000D0E03C0DBFF2D0E08D0030EDBA202D06F
:100660002B0E03D0DBA408D0200EF36E170EF3CFB1
:10067000DBFF150EDB2A02D0170EDB6A050EDB50FE
:1006800003E1B7D901E189D0680E256E4C0E266EC4
:10069000000E276E070EDBCF28F0296A2A6A2B6A24
:1006A00028C00BF029C00CF02AC00DF02BC00EF0B2
:1006B000D3D9CBEC25F025500024F36E2650012031
:1006C000F46E27500220F86EF4CFF7FFF3CFF6FF59
:1006D0000800090EF5CFDBFF580EDF5C0FE1610E5D
:1006E000F36E090E7BD90AE3200E256E090EDBCFCF
:1006F000E7FF2550E75E090EE7CFDBFF070EDBCFF4
:1007000025F0266A276A286A0FDA25C00BF026C072
:100710000CF027C00DF028C00EF0EECF04F0EECFA5
:1007200005F0EECF06F0EFCF07F0CBEC25F007C0D9
:10073000EDFF06C0EDFF05C0EDFF04C0EFFF390E71
:10074000DBCFE9FFDB063A0EDBCFEAFF01E2DB0697
:10075000090EDBCFEFFF150EDB2A4BD995E1030E17
:10076000DBA61DD06F0EDF5C06E1C1D918E3150EC4
:10077000DB285BDA14D0780EDF5C09E0580EDF5C12
:1007800006E0620EDF5C03E0420EDF5C08E1020E71
:10079000F36E160EF3CFDBFF02D0150EDB6A030EED
:1007A000DB50100B0EE0040EDBCF25F0050EDB5006
:1007B000D880255406E2060EDB5003E1040EDB5020
:1007C00034DA95D90AE2050EDBCFE7FF150EDB50D0
:1007D000E75E050EE7CFDBFF02D0050EDB6A040EF5
:1007E000DBCF25F0160E45D9D880255414E2160E1D
:1007F000DBCFE6FF150EDBCFE6FF040EDBCFE6FF17
:10080000050EDB50E552E75CE552D880E754E5522F
:10081000D880E7545FD9030EDB50010B0BE1080EC3
:10082000DB5008E0B2D801E08DD0080EDB50BED816
:10083000080EDB6A170EDB5007E088D9170EF1D9D6
:1008400003E1261C01E17ED0160EDB5016E07ED9B6
:10085000300EE66E9FD802E1261C74E077D9DFCF18
:10086000E6FF27EC25F0E552E552E552F4CF26F0FD
:100870000001F31C02E1261C65E0050EDBCF25F02C
:10088000160EDB50D880255409E2050EDBCFE7FFBA
:10089000160EDB50E75E050EE7CFDBFF300EE66E8F
:1008A000050ECBD94FE1390EDB2ADBCFE9FF3A0E3B
:1008B00001E3DB2ADBCFEAFF090EEFCFDBFFDB50E2
:1008C0000EE044D9090EADD902E1261C3BE0390EF9
:1008D000DB2ADBCFE9FF3A0EEDE3DB2AEBD755D875
:1008E00031E1160EDBCFE6FF080EC3D8E552E72450
:1008F0005DD82ED0070EDB50030A1CE0010A14E07D
:10090000030A07E07BD9DBCFEEFF020EDBCFEDFF62
:100910001FD0F5D82A6A28AE02D029682A682CD8B8
:10092000BCD82AC0EEFF14D0EAD828BE296824D843
:10093000B4D80ED063D9DBCFEFFF0AD07BD905E165
:10094000261C03E1F368F46810D0FCD801E3DB2A2D
:1009500079D947EF00F0010EDBCF25F0020EDBCF97
:1009600026F025C0F3FF26C0F4FF3B0EE15C02E257
:10097000E16AE552E16ECBD029D9020EADEF05F068
:1009800061D90800F550DF6E1200200EE66E080EE9
:100990001DEF06F027EC25F0E552E552E552F3CFC6
:1009A00025F0F4CF26F00001F31C1200256E266A14
:1009B000D950010F4DD92550EE262650ED221200B8
:1009C000295E000E2A5AF70E29C0DBFFF80E2AC056
:1009D000DBFF29C0E9FF2AC0EAFF1200DBCFF4FFEA
:1009E000F350F45C1200DB50E76E040EE7CFDBFF40
:1009F00012000A0EDBCF25F00B0EDBCF26F00C0E1B
:100A0000DBCF27F00D0EDBCF28F025502610271066
:100A100028101200130EEECFDBFF140EEDCFDBFF1C
:100A2000130EDBCF25F0140EDBCF26F00001800E75
:100A300026141200F70EDBCF29F0F80EDBCF2AF0D8
:100A40001200050EDB50E66ED950130F01D9E552A6
:100A5000E750EE6EED6A12000A0EDBCF04F00B0ECB
:100A6000DBCF05F00C0EDBCF06F00D0EDBCF07F071
:100A70001200DBCFE6FF150EDBCFE6FF050EDB50E5
:100A8000E552E724E552E7241200DB50CED8010EF0
:100A9000F36E060EF3CFDBFF1200EE50EFCFEAFF4E
:100AA000E96E27C0EEFF28C0EEFF29C0EEFF12005E
:100AB000D9CFE6FFDACFE6FFE1CFD9FFE2CFDAFF09
:100AC0001200DFCFE6FFE66AB9EC25F0E552E55209
:100AD000F3501200E76E080EE7CFDBFF1200EECFF7
:100AE00025F0EECF26F0EFCF27F0286A1200050E92
:100AF000DBCF25F0150EDB50D88025541200010EF7
:100B0000DBCF27F0020EDBCF28F0296A1200E55276
:100B1000E5CFDAFFE7CFD9FF12000A0E25C0DBFFD1
:100B20000B0E26C0DBFF1200D9500A0F28EF06F08B
:100B3000F36E070EF3CFDBFF1200EECF25F0EFCF01
:100B400026F01200010EDB2A020E1200FC0EDBCF93
:100B5000E6FFFD0EDBCFE6FF1200255E000E265AF3
:100B6000F70E25C0DBFFF80E26C0DBFF25C0E9FF2E
:100B700026C0EAFF1200DA20EA6EEF2AEECFF6FF77
:100B8000000EEF22EECFF7FFEF22EECFF8FF1200BC
:100B9000040EDBCFE6FF130EDB50E552E75C9ADF75
:100BA000DB5004DF060EDB501200090EDB500A0D8D
:100BB000F350DF24D00FE76E090EE7CFDBFFC0EF65
:100BC00004F0DB50F36E050EEEEF04F0F70EDBCF12
:100BD00025F0F80EDBCF26F01200DFCFE6FFCAEFDC
:100BE00004F028DF030EECDE6FEF05F01CEC00F0E4
:100BF000E552E552E552E55200091200BDDEEE5025
:100C0000EFCFEAFFE96E010E1200130EDB50F36E18
:100C1000040EEEEF04F0040EDB50F36E090EEEEF5F
:100C200004F0DBCFE6FFCAEF04F0E76E050EE7CF76
:100C3000DBFF12008BDFEDEF05F0DBCFE6FF86DF99
:100C4000F6EF05F0D950F90FE96EFF0EBBEF05F096
:0A0C5000E96E000EDA20EA6E1200D1
:060C5A00DACFE4FFE652D0
:100C6000E552E5CFDAFF1100D8CFE4FFE0CFE4FF93
:100C7000E46EDACFE4FFE652E552E5CFDAFFE55065
:100C8000E5CFE0FFE5CFD8FF100045D8B6EC23F064
:100C90000101E26BE36B010EE46FB050E66EE66AB1
:100CA000AF50E66EE66A1C0EE66E450EE66E290E45
:100CB000256E450E266E276A25C0E6FFE66E27C024
:100CC000E6FF000EE66E010EE66E82EC24F0286E62
:100CD0000B0EE15E2850000EE66E010EE66EFDEC96
:100CE00023F0E552E552400EE66EE66AE66A800EB3
:100CF000E66E010EE66E48EC23F0256E050EE15E11
:100D000025500101800EC06F010EC16FF6EC12F08C
:100D1000BAEC21F0FBD70F0EC11206D86AEC12F024
:100D2000080E146E92EF1BF00101EC6BEB6B010EE1
:100D3000EA6F12000501F651F71104E1100EF66F8B
:100D4000270EF76FF607000EF75B6DA207D0F6517E
:100D5000F7112EE18B7C8BBC13D027D0020172518E
:100D600002E18B9C22D0720502E18B8C09D0020E2D
:100D7000725D02E18B8C19D0040E725D03E18B9CD5
:100D80008B8E1200100E725D06E10501F651F7110F
:100D90000FE18B7C0AD0200E725D0AE10501F6514D
:100DA000F71106E18B7C8BAC02D08B9E12008B8EF0
:100DB0001200120012000101EB5109E1EC5102E0B6
:100DC000EC071200010EEB6F640EEC6F1200EC5199
:100DD00001E0EC071200120056EF1FF01200A4EF22
:100DE0001FF0020196051EE1020197051BE1E2DFFB
:100DF0006D920201976B0101100EED6F0E0EEE6FFA
:100E0000ED07000EEE5BED51EE11FAE16D84080E78
:100E1000ED6F070EEE6FED07000EEE5BED51EE117C
:100E2000FAE16D941200D9CFE6FFE1CFD9FFFD0EB4
:100E3000DBCF06F0FE0EDBCF07F0050E061801E152
:100E4000075036E0E868061802E17F0E07182FE029
:100E5000030E061801E1075028E0020E061801E112
:100E6000075021E0010E061801E107501AE0740E48
:100E7000061801E1075013E0750E061801E107504E
:100E80000CE0730E061801E1075005E0720E06181B
:100E90000FE107500DD08FDF0BD08BDF09D08ADF39
:100EA00007D09DDF05D09ADF03D096DF01D093DF16
:0A0EB000010EE552E7CFD9FF120052
:060EBA00FF0EE3CFEAFF8A
:100EC000E552FF0EE3CFE9FFE552E66AE66AD9CFC5
:100ED000E6FFDACFE6FFFC0EE124D96EFF0EE2203A
:100EE000DA6EE66AE66AE66A200EEF5C06E0090E54
:100EF000EF5C03E0EF6603D03FD0EE50F5D72D0E48
:100F0000EF5C03E1FF0EE32A03D02B0EEF5C01E15F
:100F1000EE502F0EEF6424D03A0EEF6021D0D8901F
:100F2000F90EE336FA0EE336FD0EDECFE3FFFE0EDA
:100F3000DDCFE3FFD890F90EE336FA0EE336D89012
:100F4000F90EE336FA0EE336FD0EE350DE26FE0E12
:100F5000E350DD22300EEE5CDE26000EDD22D9D716
:100F6000FF0EE3CFE8FFE85207E0F90EE31EE32AA5
:100F7000FA0ED8B4E306E31EE552E552E552FF0E41
:100F8000E3CFDAFFE552FF0EE3CFD9FFE552E1CF21
:100F9000E9FFE2CFEAFFED52ED52EECFF3FFEFCFE4
:040FA000F4FF120048
:0C0FA40007C013F006C012F006500D024A
:100FB000F4CF05F0F3CF04F007500E02F4CF07F0A2
:100FC000F3CF06F00D02F3500526F4500622E86A2E
:100FD000072212500E02F3500526F4500622E86A4A
:100FE00007220EAEF8EF07F01250065E1350075AB4
:0E0FF00013AE000C0D50065E0E50075A000C9A
:020FFE001200DF
:06100000FFEF25F01200D5
:02100600FFFFEA
:061008002DEF06F01200BE
:021016000001D7
:0610180034EF06F01200A7
:02101E00D9CF28
:10102000E6FFE1CFD9FF0D0EE126FD0EDBCF06F086
:10103000FE0EDBCF07F0090E06C0DBFF0A0E07C06D
:10104000DBFF070EDB6A080EDB6A050EDB6A060EA5
:10105000DB6A050EDBCF25F0060EDBCF26F0FB0E9C
:10106000DBCF27F0FC0EDBCF28F02750255C285083
:10107000265801E36AD2090EDBCFE9FFDB2A0A0E0C
:10108000DBCFEAFF01E3DB2AEFCFDFFF0501EE5103
:10109000030A01E1E8D1010A01E1CAD1030A01E131
:1010A000BBD1010A01E03FD21B0EDF5C02E1010E61
:1010B00004D02B0EDF5C03E1020EEE6F3FD20D0E6B
:1010C000DF5C04E00A0EDF5C01E0FBD0F90EDBCF51
:1010D00025F0FA0EDBCF26F00101C051255CC1518D
:1010E000265801E32BD214A61FD00401320EC06F84
:1010F000050EC16F3F0EC26F550EC36F200E050166
:10110000EF250401C46FC56BBEEC1BF00A0EE66E42
:1011100029EC26F0E55215EC21F0010EE66E46ECC6
:101120001FF0E552BEEC1BF0030EDB6A040EDB6A17
:10113000F90EDBCF06F0FA0EDBCF07F00B0E06C080
:10114000DBFF0C0E07C0DBFF400EE66EE66AE66AC8
:10115000C00EE66E040EE66E48EC23F0256E050E1A
:10116000E15E25500401200EC06F0B0EDBCF25F091
:101170000C0EDBCF26F00101C051255CC151265871
:1011800026E20B0EDBCFE9FF0C0EDBCFEAFFEF50C0
:10119000E66E020EE76E030EDBCFE9FF040EDBCF37
:1011A000EAFFE750E926000EEA22C00EE926040E07
:1011B000EA22E552E750EF6E0B0EDB2A0C0E01E33C
:1011C000DB2A030EDB2A040ED0E3DB2ACED705018F
:1011D000F05102E0F00517E1020EE76E030EDBCFDF
:1011E000E9FF040EDBCFEAFFE750E926000EEA2212
:1011F000C00EE926040EEA220D0EEF6E030EDB2A66
:10120000040E01E3DB2AF05103E0020EF05D17E16A
:10121000020EE76E030EDBCFE9FF040EDBCFEAFF21
:10122000E750E926000EEA22C00EE926040EEA2263
:101230000A0EEF6E030EDB2A040E01E3DB2A030E17
:10124000DBCF25F0040EDBCF26F0020E25240401AF
:10125000C16FF90EDBCFC0F1FA0EDBCFC1F1186A16
:10126000BEEC1BF00A0EE66E29EC26F0E55215ECFA
:1012700021F015EC21F0010E14141BE0080E1414DB
:1012800018E00401320EC06F050EC16F3F0EC26F31
:10129000550EC36F400E0501EF250401C46FC56BE9
:1012A000BEEC1BF00A0EE66E1BEC26F0E55215ECC8
:1012B00021F0010EF36E070EF3CFDBFF080EDB6AA1
:1012C0003DD1F90EDB500101C05D256EFA0EDB50F9
:1012D000C1590001266ED890E85004E63D0E255C09
:1012E000000E265801E21FD114A61FD00401320EB1
:1012F000C06F050EC16F3F0EC26F550EC36F200E3B
:101300000501EF250401C46FC56BBEEC1BF00A0E8E
:10131000E66E29EC26F0E55215EC21F0010EE66EA2
:1013200046EC1FF0E552BEEC1BF0030EDB6A040E28
:10133000DB6AF90EDBCF06F0FA0EDBCF07F00B0EFF
:1013400006C0DBFF0C0E07C0DBFF400EE66EE66A50
:10135000E66AC00EE66E040EE66E48EC23F0256EDB
:10136000050EE15E25500401200EC06F0B0EDBCF91
:1013700025F00C0EDBCF26F00101C051255CC151D8
:10138000265826E20B0EDBCFE9FF0C0EDBCFEAFF7F
:10139000EF50E66E020EE76E030EDBCFE9FF040EA0
:1013A000DBCFEAFFE750E926000EEA22C00EE9266D
:1013B000040EEA22E552E750EF6E0B0EDB2A0C0E0C
:1013C00001E3DB2A030EDB2A040ED0E3DB2ACED7AF
:1013D000030EDBCF25F0040EDBCF26F0020E252412
:1013E0000401C16FF90EDBCFC0F1FA0EDBCFC1F102
:1013F000186ABEEC1BF00A0EE66E29EC26F0E552E8
:1014000015EC21F015EC21F0010EF36E070EF3CF71
:10141000DBFF080EDB6A87D0DF50C0C1E9FFC1C126
:10142000EAFFEF6E0101C02B000EC123182A6DD018
:101430002B0EDF5C16E1030EEE6F320EE66EE66AEF
:10144000E66A400EE66E020EE66E48EC23F0256E6C
:10145000050EE15E25500001400EFB6F020EFC6F91
:101460006DD0EE6B60D00D0EDF5C03E00A0EDF5C2A
:101470004FE1FBC0E9FFFCC0EAFFEF6AFBC025F0CB
:10148000FCC026F0400E255E020E265A25C0E6FF5F
:1014900026C0E6FFF50EDBCFE6FFF60EDBCFE6FF5C
:1014A000400EE66E020EE66E64D8276E060EE15E12
:1014B0002750DE52F3CFDEFFF4CFDDFFDD52D950EF
:1014C000010FE96EDACFEAFFEE50ED1014E10101F1
:1014D000C0C1E9FFC1C1EAFFC02B000EC1232B0E22
:1014E000EF6EC0C1E9FFC1C1EAFFC02B000EC123EE
:1014F0002B0EEF6E0AD0F50EDBCFE6FFF60EDBCF3C
:10150000E6FF94EC20F0E552E5520501EE6B16D0B3
:10151000DF50FBC0E9FFFCC0EAFFEF6E0001FB2BD0
:10152000000EFC230BD0DF50C0C1E9FFC1C1EAFFB0
:10153000EF6E0101C02B000EC123182A050EDB2A15
:10154000060E01E286D5DB2A84D5070EDBCF25F017
:10155000080EDBCF26F025C0F3FF26C0F4FF0D0EEA
:10156000E15C02E2E16AE552E16EE552E7CFD9FFC4
:101570001200D9CFE6FFE1CFD9FF530EE126F90ED5
:10158000DBCF25F0FA0EDBCF26F0263406E225501D
:101590003208000E265401E2D2D1FD0EDBCF06F058
:1015A000FE0EDBCF07F0DE5206C0DEFF07C0DDFF18
:1015B000DD52320EE66EE66AE66AD950050FE66E37
:1015C000000EDA20E66E48EC23F0256E050EE15E93
:1015D00025504B0EDB6A4C0EDB6A4B0EDBCF25F041
:1015E0004C0EDBCF26F0F90EDBCF27F0FA0EDBCF67
:1015F00028F026502818E8AE02D0283404D027500E
:10160000255C2850265829E2010EDBCFE9FFDB2AB2
:10161000020EDBCFEAFF01E3DB2AEFCFDFFF0D0E87
:10162000DF5C1BE00A0EDF5C18E0200EDF5C15E0DB
:10163000D950050F256EDACF26F04B0EDB5025244E
:10164000E96E4C0EDB50DA20EA6EDFCFEFFF4B0E77
:10165000DB2A4C0EC2E3DB2AC0D7D950030FE96E58
:10166000DACFEAFFE90EEE6E050EED6E200EDF5CBE
:1016700001E08DD04B0EDBCF25F0DB2A4C0EDBCF0B
:1016800026F001E3DB2AF90EDBCF27F0FA0EDBCFE1
:1016900028F026502818E8AE02D0283404D027506D
:1016A000255C2850265843E2010EDBCFE9FF020EED
:1016B000DBCFEAFFEFCFDFFF200EDF5CDBE0DFCF29
:1016C000E6FFE66AA1EC25F0E552E552F3CF27F0FC
:1016D000F4CF28F0F3CFE6FFF4CFE6FFDFCFE6FF4D
:1016E000E66AB9EC25F0E552E552E552E7CF28F07D
:1016F000E552E7CF27F02750F310256E2850F4105D
:10170000266E255026100DE0010EDBCF06F0020EEE
:10171000DBCF07F0030E06C0DBFF040E07C0DBFFC4
:1017200006D0010EDB2A020EA5E3DB2AA3D74B0E5F
:10173000DBCF25F0DB2A4C0EDBCF26F001E3DB2AE2
:10174000F90EDBCF27F0FA0EDBCF28F02650281851
:10175000E8AE02D0283404D02750255C2850265803
:1017600016E2010EDBCFE9FF020EDBCFEAFFEFCF7F
:10177000DFFF0D0EDF5C0BE00A0EDF5C08E0DF50E0
:1017800006E0010EDB2A020ED2E3DB2AD0D74B0E95
:10179000DBCF06F04C0EDBCF07F04F0E06C0DBFFB1
:1017A000500E07C0DBFF4B0EDB6A4C0EDB6A4B0EA4
:1017B000DBCF25F04C0EDBCF26F0D890265004E688
:1017C000640E255C000E265801E3B9D04B0EDBCF2A
:1017D000E9FF4C0EDBCFEAFFD890E936EA36D89025
:1017E000E936EA36910EE926050EEA22020EE926CE
:1017F000000EEA22EE50ED1001E1A1D04B0EDBCF3E
:10180000E9FF4C0EDBCFEAFFD890E936EA36D890F4
:10181000E936EA36910EE926050EEA22EECF25F0EA
:10182000EFCF26F0276A25C0E6FF26C0E6FF27C0D7
:10183000E6FF62EC23F0E552E552E552510E05C099
:10184000DBFF520E06C0DBFF510EDBCFE6FF520E70
:10185000DBCFE6FFFD0EDBCFE6FFFE0EDBCFE6FFC4
:101860004B0EDBCFE9FF4C0EDBCFEAFFD890E93619
:10187000EA36D890E936EA36910EE926050EEA22D4
:10188000EECF25F0EFCF26F0276A25C0E6FF26C071
:10189000E6FF27C0E6FF87EC23F0286E070EE15E27
:1018A0002850000945E14B0EDBCFE9FF4C0EDBCFA2
:1018B000EAFFD890E936EA36D890E936EA36910E52
:1018C000E926050EEA22020EE926000EEA22EECFF4
:1018D00025F0EFCF26F0030EDBCFE6FF040EDBCFC3
:1018E000E6FFFB0EDBCFE6FFFC0EDBCFE6FFFD0ED7
:1018F000DBCFE6FFFE0EDBCFE6FF04D026C0FAFF0B
:101900002550F96EFBDF276E060EE15E27504D0E67
:10191000F3CFDBFF4E0EF4CFDBFF4F0EDBCF25F016
:10192000500EDBCF26F025C0F3FF26C0F4FF09D010
:101930004B0EDB2A4C0E01E23AD7DB2A38D7F36A8A
:10194000F46A530EE15C02E2E16AE552E16EE552AF
:10195000E7CFD9FF1200D9CFE6FFE1CFD9FFF90ECB
:10196000DBCF25F0FA0EDBCF26F0E90E25181EE1BD
:10197000050E26181BE10501EF51E66EE66A1B0E07
:10198000256E460E266E276A25C0E6FFE66E27C046
:10199000E6FFFB0EDBCFE6FFFC0EDBCFE6FF82ECC3
:1019A00024F0286E070EE15E285013D0F90EDBCF2D
:1019B000E6FFFA0EDBCFE6FF5DEC07F0E552E552FD
:1019C000F3CFEFF5FB0EDBCFE9FFFC0EDBCFEAFF39
:1019D000EF6A010EF36EF46AE552E7CFD9FF120009
:1019E000D9CFE6FFE1CFD9FF020EE126DE6ADD6A3C
:1019F000F90EDBCF25F0FA0EDBCF26F0E90E251825
:101A00002CE1050E261829E1010E141402E1000E46
:101A100001D0010E256E266A25BE266825C0DEFF90
:101A200026C0DDFFDECFE6FFDDCFE6FF1B0E256E15
:101A3000460E266E276A25C0E6FFE66E27C0E6FF43
:101A4000FB0EDBCFE6FFFC0EDBCFE6FF82EC24F0E3
:101A5000286E070EE15E285024D0F90EDBCFE6FF9A
:101A6000FA0EDBCFE6FF5DEC07F0E552E552F3CF6F
:101A7000DEFFF4CFDDFFD9CFE9FFDACFEAFF010EB9
:101A8000EE1805E1ED5003E1010E141002D0FE0E38
:101A90001414146EFB0EDBCFE9FFFC0EDBCFEAFF64
:101AA000EF6A010EF36EF46A020EE15C02E2E16A93
:101AB000E552E16EE552E7CFD9FF1200D9CFE6FF3C
:101AC000E1CFD9FFF50E256E450E266E276A25C09B
:101AD000E6FFE66E27C0E6FFFB0EDBCFE6FFFC0E5F
:101AE000DBCFE6FF82EC24F0286E050EE15E285085
:101AF000010EF36EF46AE552E7CFD9FF1200D9CF99
:101B0000E6FFE1CFD9FF1DEC1FF0FB0EDBCFE9FFB5
:101B1000FC0EDBCFEAFFEF6A010EF36EF46AE552CA
:101B2000E7CFD9FF1200D9CFE6FFE1CFD9FFBB0E37
:101B3000E66E450EE66EC70E256E450E266E276ACA
:101B400025C0E6FFE66E27C0E6FFFB0EDBCFE6FF13
:101B5000FC0EDBCFE6FF82EC24F0286E070EE15E80
:101B60002850010EF36EF46AE552E7CFD9FF120058
:101B7000D9CFE6FFE1CFD9FF0401320EC06F060EC8
:101B8000C16F3F0EC26F550EC36F200E0501EF25CA
:101B90000401C46F040EC56FC66BBEEC1BF0FB0ED8
:101BA000DBCFE9FFFC0EDBCFEAFFEF6A010EF36E3D
:101BB000F46AE552E7CFD9FF1200D9CFE6FFE1CFB3
:101BC000D9FF020EE126DE6ADD6AF90EDBCF25F0D1
:101BD000FA0EDBCF26F0E90E25182CE1050E2618AB
:101BE00029E1020E141402E1000E01D0010E256E4F
:101BF000266A25BE266825C0DEFF26C0DDFFDECFB3
:101C0000E6FFDDCFE6FF1B0E256E460E266E276A29
:101C100025C0E6FFE66E27C0E6FFFB0EDBCFE6FF42
:101C2000FC0EDBCFE6FF82EC24F0286E070EE15EAF
:101C3000285024D0F90EDBCFE6FFFA0EDBCFE6FF0B
:101C40005DEC07F0E552E552F3CFDEFFF4CFDDFFA8
:101C5000D9CFE9FFDACFEAFF010EEE1805E1ED502A
:101C600003E1020E141002D0FD0E1414146EFB0ECC
:101C7000DBCFE9FFFC0EDBCFEAFFEF6A010EF36E6C
:101C8000F46A020EE15C02E2E16AE552E16EE552BD
:101C9000E7CFD9FF1200D9CFE6FFE1CFD9FFF90E88
:101CA000DBCF25F0FA0EDBCF26F0E90E25181EE17A
:101CB000050E26181BE10501F051E66EE66A1B0EC3
:101CC000256E460E266E276A25C0E6FFE66E27C003
:101CD000E6FFFB0EDBCFE6FFFC0EDBCFE6FF82EC80
:101CE00024F0286E070EE15E285013D0F90EDBCFEA
:101CF000E6FFFA0EDBCFE6FF5DEC07F0E552E552BA
:101D0000F3CFF0F5FB0EDBCFE9FFFC0EDBCFEAFFF4
:101D1000EF6A010EF36EF46AE552E7CFD9FF1200C5
:101D2000D9CFE6FFE1CFD9FF020EE126DE6ADD6AF8
:101D3000F90EDBCF25F0FA0EDBCF26F0E90E2518E1
:101D40002CE1050E261829E1040E141402E1000E00
:101D500001D0010E256E266A25BE266825C0DEFF4D
:101D600026C0DDFFDECFE6FFDDCFE6FF1B0E256ED2
:101D7000460E266E276A25C0E6FFE66E27C0E6FF00
:101D8000FB0EDBCFE6FFFC0EDBCFE6FF82EC24F0A0
:101D9000286E070EE15E285024D0F90EDBCFE6FF57
:101DA000FA0EDBCFE6FF5DEC07F0E552E552F3CF2C
:101DB000DEFFF4CFDDFFD9CFE9FFDACFEAFF010E76
:101DC000EE1805E1ED5003E1040E141002D0FB0EF5
:101DD0001414146EFB0EDBCFE9FFFC0EDBCFEAFF21
:101DE000EF6A010EF36EF46A020EE15C02E2E16A50
:101DF000E552E16EE552E7CFD9FF1200D9CFE6FFF9
:101E0000E1CFD9FFF90EDBCF25F0FA0EDBCF26F0BC
:101E1000E90E25181EE1050E26181BE10501F151FA
:101E2000E66EE66A1B0E256E460E266E276A25C0F4
:101E3000E6FFE66E27C0E6FFFB0EDBCFE6FFFC0EFB
:101E4000DBCFE6FF82EC24F0286E070EE15E28501F
:101E500013D0F90EDBCFE6FFFA0EDBCFE6FF5DEC29
:101E600007F0E552E552F3CFF1F5FB0EDBCFE9FFCA
:101E7000FC0EDBCFEAFFEF6A010EF36EF46AE55267
:101E8000E7CFD9FF1200D9CFE6FFE1CFD9FFE66A4D
:101E900046EC1FF0E552FB0EDBCFE9FFFC0EDBCF7B
:101EA000EAFFEF6A010EF36EF46AE552E7CFD9FF5D
:101EB0001200D9CFE6FFE1CFD9FF020EE126DE6A9C
:101EC000DD6AF90EDBCF25F0FA0EDBCF26F0E90E46
:101ED00025182CE1050E261829E1100E141402E134
:101EE000000E01D0010E256E266A25BE266825C08B
:101EF000DEFF26C0DDFFDECFE6FFDDCFE6FF1B0EF7
:101F0000256E460E266E276A25C0E6FFE66E27C0C0
:101F1000E6FFFB0EDBCFE6FFFC0EDBCFE6FF82EC3D
:101F200024F0286E070EE15E285024D0F90EDBCF96
:101F3000E6FFFA0EDBCFE6FF5DEC07F0E552E55277
:101F4000F3CFDEFFF4CFDDFFD9CFE9FFDACFEAFF31
:101F5000010EEE1805E1ED5003E1100E141002D051
:101F6000EF0E1414146EFB0EDBCFE9FFFC0EDBCF7B
:101F7000EAFFEF6A010EF36EF46A020EE15C02E220
:101F8000E16AE552E16EE552E7CFD9FF1200D9CF01
:101F9000E6FFE1CFD9FF020EE126DE6ADD6AF90E27
:101FA000DBCF25F0FA0EDBCF26F0E90E25182CE169
:101FB000050E261829E1080E141402E1000E01D0C6
:101FC000010E256E266A25BE266825C0DEFF26C0C6
:101FD000DDFFDECFE6FFDDCFE6FF1B0E256E460EF2
:101FE000266E276A25C0E6FFE66E27C0E6FFFB0ED9
:101FF000DBCFE6FFFC0EDBCFE6FF82EC24F0286EA1
:10200000070EE15E285029D0F90EDBCFE6FFFA0E6D
:10201000DBCFE6FF5DEC07F0E552E552F3CFDEFFE4
:10202000F4CFDDFFD9CFE9FFDACFEAFF010EEE18DA
:1020300006E1ED5004E1080E1410146E07D0F70EFF
:102040001414146EE66A46EC1FF0E552FB0EDBCF6B
:10205000E9FFFC0EDBCFEAFFEF6A010EF36EF46AD4
:10206000020EE15C02E2E16AE552E16EE552E7CF81
:10207000D9FF1200D9CFE6FFE1CFD9FFF90EDBCFB0
:1020800025F0FA0EDBCF26F0E90E251806E1050E45
:10209000261803E10501F46B31D0030EE66EE66A03
:1020A000F90EDBCFE6FFFA0EDBCFE6FF7E0E256EE4
:1020B000460E266E276A25C0E6FFE66E27C0E6FFBD
:1020C00087EC23F0286E070EE15E2850000903E13B
:1020D0000501010E12D0F90EDBCFE6FFFA0EDBCFC1
:1020E000E6FF5DEC07F0E552E552F3CFE7F10101C1
:1020F000E751000803E20501020EF46F0401320EFD
:10210000C06F050EC16F3F0EC26F550EC36F400EFC
:102110000501EF250401C46FC56BBEEC1BF0FB0E7F
:10212000DBCFE9FFFC0EDBCFEAFFEF6A010EF36EB7
:10213000F46AE552E7CFD9FF1200D9CFE6FFE1CF2D
:10214000D9FFF90EDBCF25F0FA0EDBCF26F0E90E32
:1021500025181EE1050E26181BE1F2C5E6FFF3C5A2
:10216000E6FF1B0E256E460E266E276A25C0E6FF8B
:10217000E66E27C0E6FFFB0EDBCFE6FFFC0EDBCFF3
:10218000E6FF82EC24F0286E070EE15E285015D0A1
:10219000F90EDBCFE6FFFA0EDBCFE6FF5DEC07F0D2
:1021A000E552E552F3CFF2F5F4CFF3F5FB0EDBCFBA
:1021B000E9FFFC0EDBCFEAFFEF6A010EF36EF46A73
:1021C000E552E7CFD9FF1200D9CFE6FFE1CFD9FF23
:1021D000400EE66EE66AE66A800EE66E010EE66E78
:1021E00048EC23F0256E050EE15E25500501EE6BEF
:1021F000090E146E0501F06B05012A0EF16F050141
:102200002C0EF26F010EF36F0501F46FD950FB0F26
:10221000E96EDACFEAFF800EEE6E010EED6E176A00
:10222000186A010EF36EF46AE552E7CFD9FF120087
:10223000D9CFE6FFE1CFD9FF020EE1260501EF512C
:10224000DE6EDD6AFB0EDBCFE9FFFC0EDBCFEAFFC3
:10225000EF6AF90EDBCF25F0FA0EDBCF26F0E90EA0
:10226000251802E1050E26180EE0F90EDBCFE6FF79
:10227000FA0EDBCFE6FF5DEC07F0E552E552F3CF57
:10228000DEFFF4CFDDFF0401320EC06F060EC16F1A
:102290003F0EC26F350EC36F180EC46FDECF25F030
:1022A000DDCF26F0400E2524C56FBEEC1BF072EC8E
:1022B0001DF0175000081BE204014051E66EE66A6B
:1022C0001B0E256E460E266E276A25C0E6FFE66EBB
:1022D00027C0E6FFFB0EDBCFE6FFFC0EDBCFE6FF01
:1022E00082EC24F0286E070EE15E2850176A040184
:1022F000320EC06F050EC16F190EC26F5F0EC36F35
:102300003F0EC46FC56BBEEC1BF0010EF36EF46A9A
:10231000020EE15C02E2E16AE552E16EE552E7CFCE
:10232000D9FF1200D9CFE6FFE1CFD9FF020EE12697
:10233000010EDE6EDD6A80A402D0DE6ADD6ADECFC9
:10234000E6FFDDCFE6FF1B0E256E460E266E276AE2
:1023500025C0E6FFE66E27C0E6FFFB0EDBCFE6FFFB
:10236000FC0EDBCFE6FF82EC24F0286E070EE15E68
:102370002850010EF36EF46A020EE15C02E2E16A9B
:10238000E552E16EE552E7CFD9FF1200D9CFE6FF63
:10239000E1CFD9FF020EE1260501EF51DE6EDD6AC5
:1023A000FB0EDBCFE9FFFC0EDBCFEAFFEF6AF90E95
:1023B000DBCF25F0FA0EDBCF26F0E90E251802E17F
:1023C000050E26180EE0F90EDBCFE6FFFA0EDBCF86
:1023D000E6FF5DEC07F0E552E552F3CFDEFFF4CF08
:1023E000DDFF0401320EC06F060EC16F3F0EC26FDB
:1023F000550EC36FDECF25F0DDCF26F0200E25244D
:10240000C46F080EC56FC66BBEEC1BF0010EF36EF9
:10241000F46A020EE15C02E2E16AE552E16EE55225
:10242000E7CFD9FF1200D9CFE6FFE1CFD9FFF90EF0
:10243000DBCF25F0FA0EDBCF26F0E90E25181EE1E2
:10244000050E26181BE10501F551E66EE66A1B0E26
:10245000256E460E266E276A25C0E6FFE66E27C06B
:10246000E6FFFB0EDBCFE6FFFC0EDBCFE6FF82ECE8
:1024700024F0286E070EE15E285013D0F90EDBCF52
:10248000E6FFFA0EDBCFE6FF5DEC07F0E552E55222
:10249000F3CFF5F5FB0EDBCFE9FFFC0EDBCFEAFF58
:1024A000EF6A010EF36EF46AE552E7CFD9FF12002E
:1024B000D9CFE6FFE1CFD9FFFB0EDBCFE9FFFC0E62
:1024C000DBCFEAFFEF6A010EF36EF46AE552E7CF65
:0424D000D9FF12001E
:0C24D400D9CFE6FFE1CFD9FFE652A09A75
:1024E0006A6A686A706A020EE66EE66AE66A710EE9
:1024F000E66E0F0EE66E48EC23F0256E050EE15EEB
:102500002550160E6F6E9F0E6B6E7B0E696EDF6A26
:10251000DF50256E266A0C0E255C000E265810E250
:10252000DF50040DF3CFE9FFF4CFEAFF000EE926F8
:10253000040EEA22EE6AEE6AEE6AEE6ADF2AE8D755
:102540006D8C6E6A6D986D9C68A607D068960201C6
:102550008A6B8F6B906B916BF7D70201010EA36FA3
:10256000A46FA56BA66B976BDF6A030EDF5C26E298
:10257000EA6ADF34FE0BEA36E96E800EE926020EC7
:10258000EA22EE6AED6AEA6ADF34FE0BEA36E96EA9
:102590007A0EE926020EEA22EE6AED6ADF50EA6A56
:1025A0009B0FE96E020EEA22EF6ADF50EA6A9E0F85
:1025B000E96E020EEA22EF6ADF2AD7D70201080E7F
:1025C000806F040E816F160E706E0401300E026F64
:1025D000040E036F080E016F840E006F0201736B0F
:1025E000726BE552E552E7CFD9FF1200D9CFE6FF73
:1025F000E1CFD9FFE652020172510FE16D6A696ABB
:10260000160E6F6E9F0E6B6E7B0E696E6DB602D0EE
:102610006D86FCD70201010E726F720508E16DBA7A
:1026200006D0686A696A69806988020E726F6850AC
:10263000040B06E06950040B03E06894D1EC18F039
:102640006DB258D06850010B08E06950010B05E0ED
:1026500041DF0201040E726F68906850100B06E0B3
:102660006950100B03E0BCEC18F0689868AC19D006
:1026700069AC0FD0010EE66EE66A000EE66EE66A01
:10268000730EE66EE66A13EC07F0256E060EE15E49
:102690002550689C0201A15101E0A107A15101E16F
:1026A000DFD96850200B05E06950200B02E0A3EC55
:1026B00018F06850020B13E06950020B10E0010E95
:1026C000E66EE66A000EE66EE66AE6687F0EE66E85
:1026D00013EC07F0256E060EE15E25506A6A040EC3
:1026E0000201E76E7219E8AE02D0E73402D0E7507B
:1026F000725D02E2A19A39D069A636D0DF6A040E73
:10270000DF5C32E268A630D06CCF98F202019851BB
:10271000780BE842E842E842996F689698B506D08F
:102720009951EA6A9E0FE96E020E05D09951EA6A44
:102730009B0FE96E020EEA22EF70995103E1E8EC7B
:1027400018F010D0000EE66EE66A980EE66E020EE5
:10275000E66E720EE66EE66A13EC07F0256E060E64
:10276000E15E2550DF2ACBD7A19AE552E552E7CFAB
:10277000D9FF1200D9CFE6FFE1CFD9FF020EE12643
:10278000FD0EDBA407D0E66AFE0EDBCFE6FFF7D92D
:10279000E552E552FD0EDBA208D0010EE66EFE0EFC
:1027A000DBCFE6FFECD9E552E552FE0EDB50266AA0
:1027B000700F256E0F0E262225C0DEFF26C0DDFF1E
:1027C000DECFE9FFDDCFEAFFFD0EDBCFEFFF020E2C
:1027D000E15C02E2E16AE552E16EE552E7CFD9FF42
:1027E0001200D9CFE6FFE1CFD9FF020EE126FD0EA0
:1027F000DB500AE0FE0EEA6ADB34FE0BEA36E96ED5
:10280000800EE926020E09D0FE0EEA6ADB34FE0BCA
:10281000EA36E96E7A0EE926020EEA22EECFDEFFF4
:10282000EDCFDDFFD9CFE9FFDACFEAFFEE50ED10B3
:1028300003E1F36AF46A44D0DECFE9FFDDCFEAFFBB
:10284000020EE926000EEA22FB0EDBCFEEFFFC0EA5
:10285000DBCFEDFFDECFE9FFDDCFEAFFEE52FA0E70
:10286000DBCFEFFF400EDECFE9FFDDCFEAFFE85020
:10287000EF16880EDECFE9FFDDCFEAFFE850EF125A
:10288000FD0EDB500AE0FE0EEA6ADB34FE0BEA3690
:10289000E96E800EE926020E09D0FE0EEA6ADB34EC
:1028A000FE0BEA36E96E7A0EE926020EEA22EF7492
:1028B000DECF25F0DDCF26F025C0F3FF26C0F4FFE4
:1028C000020EE15C02E2E16AE552E16EE552E7CF19
:1028D000D9FF1200D9CFE6FFE1CFD9FF020EE126E2
:1028E000FE0EDB5020E178C2E9FF79C2EAFFEE522A
:1028F000080EEF6E78C2E9FF79C2EAFF020EE92600
:10290000000EEA22300EEE6E040EED6E78C2E9FF84
:1029100079C2EAFF8C0EEF6E80C2E9FF81C2EAFF46
:10292000840EEF6E3BD0FD0EDB50E824276EFE0ECA
:10293000DB50040DF3502724040DF3CF25F0F4CF22
:1029400026F0000E2526040E262225C0DEFF26C016
:10295000DDFF840EDECFE9FFDDCFEAFFE850EF12A6
:10296000FD0EDB50E824276EFE0EDB50040DF35005
:102970002724010F040DF3CF25F0F4CF26F0000E2D
:102980002526040E262225C0DEFF26C0DDFF840E8C
:10299000DECFE9FFDDCFEAFFE850EF12020EE15C87
:1029A00002E2E16AE552E16EE552E7CFD9FF12009B
:1029B000D9CFE6FFE1CFD9FF6DA84ED0FE0EEA6A6F
:1029C000DB34FE0BEA36E96E800EE926020EEA22BF
:1029D000EE50EFCFEAFFE96E400EEE16EE6AEE6AB9
:1029E000EE6AFE0EEA6ADB34FE0BEA36E96E800E12
:1029F000E926020EEA22EE50EFCFEAFFE96EEE7C06
:102A0000FE0EEA6ADB34FE0BEA36E96E800EE9263A
:102A1000020EEA22EF74400E256EFE0EEA6ADB34E7
:102A2000FE0BEA36E96E800EE926020EEA22EE502F
:102A3000EFCFEAFFE96E2550EF16FE0EEA6ADB34AF
:102A4000FE0BEA36E96E800EE926020EEA22EE500F
:102A5000EFCFEAFFE96EEF7CE552E7CFD9FF120036
:102A60000201A3514DE1010EA36FA45149E1010EF2
:102A7000A46F020E875D0DE180C2E9FF81C2EAFF0B
:102A8000EE52EF6A80C2E9FF81C2EAFFC80EEF6E24
:102A90001200870535E19A6B76C2E9FF77C2EAFF3B
:102AA000EE52080EEF6E76C2E9FF77C2EAFF020E21
:102AB000E926000EEA22300EEE6E040EED6E76C2AE
:102AC000E9FF77C2EAFF840EEF6E010E9A6F78C2BB
:102AD000E9FF79C2EAFFEE52080EEF6E78C2E9FF15
:102AE00079C2EAFF020EE926000EEA22300EEE6EEF
:102AF000040EED6E78C2E9FF79C2EAFF800EEF6E38
:102B000012000201A56BA66B020E875D18E178C268
:102B1000E9FF79C2EAFFEE52080EEF6E78C2E9FFD4
:102B200079C2EAFF020EE926000EEA22380EEE6EA6
:102B3000040EED6E78C2E9FF79C2EAFF1DD08B5119
:102B40000401365D02018C510401375904E236C498
:102B50008BF237C48CF2CAD880C2E9FF81C2EAFF87
:102B6000020EE926000EEA22380EEE6E040EED6E1D
:102B700080C2E9FF81C2EAFFC80EEF6E1200D9CF12
:102B8000E6FFE1CFD9FF020EE126000EDE6E040E55
:102B9000DD6EFD0EDB50E824276EFE0EDB50040DCB
:102BA000F3502724040DF4CF26F0D9CFE9FFDACF74
:102BB000EAFFF350EE262650ED22DECFE9FFDDCF0F
:102BC000EAFFEF9EFD0EDB500AE1FE0EEA6ADB34FF
:102BD000FE0BEA36E96E7A0EE926020E09D0FE0EE9
:102BE000EA6ADB34FE0BEA36E96E800EE926020E55
:102BF000EA22DECFEEFFDDCFEDFFDECFE9FFDDCF56
:102C0000EAFFEF9CDECFE9FFDDCFEAFF040EE92605
:102C1000000EEA22EF8C020EE15C02E2E16AE5526C
:102C2000E16EE552E7CFD9FF12006D9802018ABF2D
:102C30002BD08FAF09D0020E876FA65101E161DF63
:102C40000201A46BA36B120078C2E9FF79C2EAFF0C
:102C5000EE52080EEF6E78C2E9FF79C2EAFF020E6B
:102C6000E926000EEA22300EEE6E040EED6E78C2FA
:102C7000E9FF79C2EAFF8C0EEF6E80C2E9FF81C2E4
:102C8000EAFF840EEF6E1200040130AF0DD0020196
:102C9000010E876FA55101E134DF0201A46BA36B24
:102CA000A25123E130EF15F00201020E876F78C2C6
:102CB000E9FF79C2EAFFEE52080EEF6E78C2E9FF33
:102CC00079C2EAFF020EE926000EEA22300EEE6E0D
:102CD000040EED6E78C2E9FF79C2EAFF840EEF6E52
:102CE000A46BA36BA25101E1BBDE1200D9CFE6FFBA
:102CF000E1CFD9FFE652080EDF6E02018B5D000EB8
:102D00008C590AE28BC2DFFF865102E1010E03D02B
:102D1000860502E1020E866FDF50266AE8508B5D61
:102D20008B6F26508C598C6F80C2E9FF81C2EAFFFD
:102D3000EE52DFCFEFFF380E946F040E956F8AB11D
:102D400018D0DF502DE088C2F6FF89C2F7FF882B2C
:102D5000000E89230800F550E66E94C2E9FF95C283
:102D6000EAFF942B000E9523E552E750EF6EDF0645
:102D7000E8D7DF5015E088C2E9FF89C2EAFF882B57
:102D8000000E8923EF50E66E94C2E9FF95C2EAFF78
:102D9000942B000E9523E552E750EF6EDF06E9D73E
:102DA000E552E552E7CFD9FF1200D9CFE6FFE1CFD8
:102DB000D9FF020EE12676C2E9FF77C2EAFFEE52A2
:102DC000EFCFDFFFDFCF25F025500201905D000E31
:102DD000915902E290C2DFFFDF50256E266AE8506B
:102DE000905D906F26509159916F010EDB6ADF5014
:102DF000F36E010EDBCFF4FFF350F45C16E2010E2C
:102E0000DB50EA6A380FE96E040EEA22EF50E66EF4
:102E10008DC2E9FF8EC2EAFF8D2B000E8E23E55294
:102E2000E750EF6E010EDB2AE2D7000ED8809055F6
:102E3000000E915527E278C2E9FF79C2EAFFEE520F
:102E4000080EEF6E78C2E9FF79C2EAFF020EE926AA
:102E5000000EEA22380EEE6E040EED6E76C2E9FF29
:102E600077C2EAFFEF50400B06E178C2E9FF79C272
:102E7000EAFFC80E05D078C2E9FF79C2EAFF880EE2
:102E8000EF6E28D078C2E9FF79C2EAFFEE52080E51
:102E9000EF6E78C2E9FF79C2EAFF020EE926000E62
:102EA000EA22300EEE6E040EED6E78C2E9FF79C2B2
:102EB000EAFF840EEF6E9251931107E005D093C2A2
:102EC000FAFF02019251F96EFADF02018F9FA251BF
:102ED00001E1C6DD020EE15C02E2E16AE552E16E6B
:102EE000E552E7CFD9FF1200D9CFE6FFE1CFD9FFF6
:102EF000E65202018A8F020EE66EE66AE66A710EFB
:102F0000E66E0F0EE66E48EC23F0256E050EE15ED0
:102F10002550300EE66EE66AE66A000EE66E040E96
:102F2000E66E48EC23F0256E050EE15E25506D8CB3
:102F3000DF6A030EDF5C10E2DF50EA6A9B0FE96E86
:102F4000020EEA22EF6ADF50EA6A9E0FE96E020E75
:102F5000EA22EF6ADF2AEDD7020EE66EE66AE66A3B
:102F6000740EE66E020EE66E48EC23F0256E050E3A
:102F7000E15E25506D9C0201080E806F040E816F8A
:102F8000000E766F040E776F76C278F2796F32C4D6
:102F900073F2735102E1100E12D0010EE66EE66A72
:102FA000730EE66E020EE66E010EE66EE66A13EC36
:102FB00007F0256E060EE15E25500201200E726FAD
:102FC000E552E552E7CFD9FF1200800E0401305DD3
:102FD00058E10201C00E8A6F04013351030A2FE049
:102FE000010A09E0030A4BE102013A0E886F480E1C
:102FF000896F120E3ED03251F66EF76AD890F636CF
:10300000F736FB0EF626480EF7220900F5CF88F2B8
:103010000A00F5CF89F2020E0201F76A8825F66EE2
:103020008951F7220800F5CF8BF2030EF76A882545
:10303000F66E8951F7220800F5CF8CF21200030ECC
:10304000325D1AE23251F66EF76AD890F636F736EC
:10305000FD0EF626480EF7220900F5CF88F20A0089
:10306000F5CF89F288C2F6FF89C2F7FF0800F55054
:1030700002018B6F8C6B120002018A6B120002013D
:103080008A6B1200D9CFE6FFE1CFD9FF020EE1260D
:103090000401386B396B30511F0B020A11E0030A2F
:1030A0000CE0010A3CE102018A8F0401388102012F
:1030B000960535E10401388332D002018A8F2FD082
:1030C00002018A8F040134BF0BD034510F0BE96E1B
:1030D000EA6AD890E936EA367A0EE926020E0AD074
:1030E00034510F0BE96EEA6AD890E936EA36800E61
:1030F000E926020EEA22EECFDEFFEDCFDDFFDECFC6
:10310000E9FFDDCFEAFFEF50800B09E0DECFE9FFFA
:10311000DDCFEAFFEF50040B02E0010E386F020131
:103120008AAF07D0380E886F040E896F8A81020E2D
:103130008B6F020EE15C02E2E16AE552E16EE5525C
:10314000E7CFD9FF120070A015D076C2E9FF77C291
:10315000EAFFEF5080080DE180C2E9FF81C2EAFF7B
:10316000EF50840806E176C2E9FF77C2EAFF8C0ED1
:10317000EF6E7090689A1200698468986D820201FF
:10318000010E976F000EE66EE66AE66EE66A750E51
:10319000E66EE66A13EC07F0256E060EE15E25503A
:1031A00012000201976B000EE66EE66AE66EE66AB2
:1031B000740EE66EE66A13EC07F0256E060EE15E0D
:1031C00025506D92699468A402D06894FCD71200CF
:1031D000D9CFE6FFE1CFD9FFE65202012D0EA16F54
:1031E000FD0E981553E17E0E9815E8407F0B040DF7
:1031F000F3CF76F2F4CF77F2000E7627040E772322
:1032000076C278F277C279F2787576C2E9FF77C232
:10321000EAFFEF503C0BE842E8420D0835E1DF6A77
:10322000080EDF5C23E276C2E9FF77C2EAFF020EF6
:10323000E926000EEA22EE50EFCFEAFFE96EEF50EA
:10324000E66EDF50EA6A300FE96E040EEA22E552BC
:10325000E750EF6E76C2E9FF77C2EAFF020EE92679
:10326000000EEA22EE2AEF22DF2ADAD776C2E9FF41
:1032700077C2EAFF020EE926000EEA22300EEE6E59
:10328000040EED6E0DD807D03AD805D0FD0E981576
:10329000040801E159D8E552E552E7CFD9FF120001
:1032A0000201866BA26BA56BA66B9A6B876B80C2C3
:1032B000E9FF81C2EAFFEF9E807580C2E9FF81C20B
:1032C000EAFFEF9E807578C2E9FF79C2EAFFEF9EC0
:1032D0008A6B8B6B8C6B8F6B906B916B8CD8000EA9
:1032E000E66EE66AE66EE66A030EE66EE66A13ECE2
:1032F00007F0256E060EE15E255015EF16F0020E62
:103300000201875D02E1D5EF16F0876B9A511AE151
:1033100078C2E9FF79C2EAFFEE52080EEF6E78C27A
:10332000E9FF79C2EAFF020EE926000EEA22300E1A
:10333000EE6E040EED6E78C2E9FF79C2EAFF8C0EE4
:10334000EF6E12009A6B1200D9CFE6FFE1CFD9FFE2
:10335000E65280C2E9FF81C2EAFFEF50400B01E074
:10336000010EDF6E02018075080E725D08E132C445
:103370006EFF6E5002E0100E01D0040E726F8705D2
:1033800026E180C2E9FF81C2EAFF020EE926000EB3
:10339000EA22380EEE6E040EED6EA8DC020E02017B
:1033A000865D06E180C2E9FF81C2EAFF840E0DD08E
:1033B000DF5006E180C2E9FF81C2EAFFC80E05D0F6
:1033C00080C2E9FF81C2EAFF880EEF6E0FD08FAF97
:1033D0000CD09251931107E005D093C2FAFF02017D
:1033E0009251F96EFADF02018F9F876BE552E55229
:1033F000E7CFD9FF120004013051600BE842E842E8
:10340000E842E842E842000901E0120031510C0AAA
:1034100050E00B0A3FE00C0A31E0010A22E00B0AFF
:103420001EE0020A1CE0030A18E0080A10E0010A84
:103430000CE00F0A08E0030A01E0120002018A8F83
:10344000080E726F1200E5EF17F074EF17F002012B
:10345000730E886F020E896F0CD042EF18F05AEF8E
:103460001AF034510201886F896B740E8827020E9E
:1034700089238A81010E8B6F8A8F120002018A8F45
:1034800004013451EA6A740FE96E020EEA2232C472
:10349000EFFF1200000EE66EE66AE66EE66A020EC6
:1034A000E66EE66A13EC07F0256E060EE15E255027
:1034B00012001200D9CFE6FFE1CFD9FF050EE126B9
:1034C0000401320510E130511F0B00090CE102012B
:1034D0008A8F030E0401315D04E10201010E966F33
:1034E00002D00201966B0401325101E011D130513A
:1034F0001F0B020801E00CD134510F0B000901E150
:1035000007D134510F0B020801E202D1200E020153
:10351000725D01E0FDD08A8F040134BF16D03451B2
:103520000F0BE96EEA6AD890E936EA367A0EE92698
:10353000020EEA22EECFDEFFEDCFDDFF34510F0B9E
:10354000EA6A9E0FE96E020E15D034510F0BE96E38
:10355000EA6AD890E936EA36800EE926020EEA22B7
:10356000EECFDEFFEDCFDDFF34510F0BEA6A9B0F8C
:10357000E96E020EEA22020EEFCFDBFFD950020FF6
:10358000E96EDACFEAFFEF50010B03E1000EDF94A2
:1035900001D0DF8434BF0BD034510F0BE96EEA6ADF
:1035A000D890E936EA367A0EE926020E0AD034516E
:1035B0000F0BE96EEA6AD890E936EA36800EE92602
:1035C000020EEA22DECFEEFFDDCFEDFF030E315D0E
:1035D00020E1DECFE9FFDDCFEAFFEF50800B11E005
:1035E00034BF07D034510F0BEA6A9E0FE96E020E0A
:1035F00006D034510F0BEA6A9B0FE96E020EEA22E5
:10360000EF82840EDECFE9FFDDCFEAFFE850EF1254
:103610007FD0DF74DECFE9FFDDCFEAFFEF50800B14
:103620001BE0DECFE9FFDDCFEAFFEF9EDECFE9FF53
:10363000DDCFEAFFEF8C020EE66EE66ADECFE6FF34
:10364000DDCFE6FF050EE66EE66A13EC07F0256EA9
:10365000060EE15E255005D0DECFE9FFDDCFEAFFA3
:10366000EF8CDF74D950020FE96EDACFEAFFEF502A
:10367000020B07E1DECFE9FFDDCFEAFFEF50800B61
:103680002BE0040134BF07D034510F0BEA6A9E0FC0
:10369000E96E020E06D034510F0BEA6A9B0FE96EF9
:1036A000020EEA22EF923B0E256EDECFE9FFDDCF60
:1036B000EAFFE850EF16020EE66EE66ADECFE6FF9E
:1036C000DDCFE6FF050EE66EE66A13EC07F0256E29
:1036D000060EE15E255007D03B0EDECFE9FFDDCFC1
:1036E000EAFFE850EF16040134510F0B266A700F01
:1036F000256E0F0E2622030E25C0DBFF040E26C00A
:10370000DBFF030EDBCFE9FF040EDBCFEAFFEF9018
:10371000050EE15C02E2E16AE552E16EE552E7CFB7
:04372000D9FF1200BB
:0C372400200E896E8B6A9468936892688E
:10373000928A176A186A196A1950256E266AD890F3
:10374000265004E6800E255C000E265809E219502A
:10375000EA6A400FE96E040EEA22EF6A192AECD7F2
:10376000196A400E195C09E21950EA6AC00FE96E45
:10377000040EEA22EF6A192AF4D71200246A020E14
:103780001A6E200E8914896E8B6A94689368DF0E16
:103790009210926E0101E26B0501F5A72ED0C1C413
:1037A00025F0266A25BE266825C0E6FF26C0E6FF6E
:1037B000C0C427F0286A27BE286827C0E6FF28C0B3
:1037C000E6FFAE0E296E450E2A6E2B6A29C0E6FF73
:1037D000E66E2BC0E6FFC20EE66E010EE66E82ECD0
:1037E00024F02C6E090EE15E2C50C20EE66E010E26
:1037F000E66EFDEC23F0E552E552320E0401C05DA9
:103800001DE19296C1C425F0266A25BE266825C012
:10381000E6FF26C0E6FFA10E276E450E286E296A38
:1038200027C0E6FFE66E29C0E6FFC20EE66E010E77
:10383000E66E82EC24F02A6E070E22D00501F5A771
:1038400021D0C1C425F0266A25BE266825C0E6FF22
:1038500026C0E6FF910EE66E450EE66E9A0E276EC6
:10386000450E286E296A27C0E6FFE66E29C0E6FFEE
:10387000C20EE66E010EE66E82EC24F02A6E090E90
:10388000E15E2A500501F5A708D0C20EE66E010ED2
:10389000E66EFDEC23F0E552E552630E245C01E197
:1038A000F4D02450620A01E1CAD0640A01E1BCD01C
:1038B000030A01E19DD0010A01E18FD0070A71E0FE
:1038C000010A07E0030A03E0010AE7E1B4D0020EAF
:1038D000DAD00501F5A72BD01A50EA6AC00FE96EBD
:1038E000040EEA22EFCF25F0266A25BE266825C001
:1038F000E6FF26C0E6FF8A0E276E450E286E296A6F
:1039000027C0E6FFE66E29C0E6FFC20EE66E010E96
:10391000E66E82EC24F02A6E070EE15E2A50C20E9B
:10392000E66E010EE66EFDEC23F0E552E552040171
:10393000C1051A5C2AE1020E141427E0320EC05DA4
:1039400024E092980501F5A720D0810EE66E450E81
:10395000E66E870E256E450E266E276A25C0E6FFA9
:10396000E66E27C0E6FFC20EE66E010EE66E82EC42
:1039700024F0286E070EE15E2850C20EE66E010E9E
:10398000E66EFDEC23F0E552E5521A50EA6AC00FEC
:10399000E96E040EEA22EF1C8A6E1A2A936A030E5D
:1039A0001ED08250020B17E11BC025F01CC026F070
:1039B0001DC027F01EC028F01B06000E1C5A1D5A01
:1039C0001E5AD8802554000E2654000E2754000E8F
:1039D000285401E262D7040E56D09490050E246E4E
:1039E000A00E1B6E860E1C6E010E1D6E1E6A55D734
:1039F0008250040B17E11BC025F01CC026F01DC02F
:103A000027F01EC028F01B06000E1C5A1D5A1E5A15
:103A1000D8802554000E2654000E2754000E28543A
:103A200001E23BD7060E2FD0936892889480040160
:103A3000C1511A5C02E2010E26D0630E24D00501AA
:103A4000F5A720D07B0EE66E450EE66E870E256E3E
:103A5000450E266E276A25C0E6FFE66E27C0E6FF04
:103A6000C20EE66E010EE66E82EC24F0286E070EA2
:103A7000E15E2850C20EE66E010EE66EFDEC23F00C
:103A8000E552E552630E246E08D7320E0401C05D84
:103A900001E19286948094689368DF0E9210926E92
:103AA0000501F5A71CD0780E256E450E266E276AF7
:103AB00025C0E6FFE66E27C0E6FFC20EE66E010EE9
:103AC000E66E82EC24F0286E050EE15E2850C20EF0
:103AD000E66E010EE66EFDEC23F0E552E5520101C3
:103AE000E26B1200D9CFE6FFE1CFD9FFE652DF6AE1
:103AF000A00E1F6E0F0E206E216A226A176A200E1A
:103B00008914896E8B6AF90E946E9368DF0E921099
:103B1000926E236A800EE66EE66AE66A400EE66EF4
:103B2000040EE66E48EC23F0256E050EE15E25508E
:103B3000630E235C01E147D11750256E266AD890A9
:103B4000265004E6800E255C000E265802E3090E7E
:103B5000236E2350090A01E131D1030A01E109D1A1
:103B60000C0A01E1E5D0030A01E1B2D0010A01E14A
:103B7000ABD0070A26E0010A10E0030A05E0010ABB
:103B8000D7E194929494D2D09482D00E1F6E070EF7
:103B9000206E216A226A020E14D182B002D0030E76
:103BA000236E1F06000E205A215A225AD8801F5415
:103BB000000E2054000E2154000E2254B9E30A0EC8
:103BC00000D1D00E1F6E070E206E216A226A9492D9
:103BD0008050080B02E1000E01D0010E166EE85075
:103BE0000CE0811CE66E1750172AEA6A400FE96E56
:103BF000040EEA22E552E750EF6E8050100B01E010
:103C0000010E156E0501F5A95CD016501FE1210EBD
:103C1000E66EE66A750E256E450E266E276A25C08D
:103C2000E6FFE66E27C0E6FFC20EE66E010EE66E08
:103C300082EC24F0286E070EE15E2850C20EE66E7C
:103C4000010EE66EFDEC23F0E552E55215501AE147
:103C5000810EE66E450EE66E811CE66EE66A6C0E1F
:103C6000256E450E266E276A25C0E6FFE66E27C044
:103C7000E6FFC20EE66E010EE66E82EC24F0286EC0
:103C8000090E15D0811CE66EE66A8A0E256E450E79
:103C9000266E276A25C0E6FFE66E27C0E6FFC20E45
:103CA000E66E010EE66E82EC24F0286E070EE15EF1
:103CB0002850C20EE66E010EE66EFDEC23F0E552D2
:103CC000E5529484040E7DD082A032D7050E79D0BF
:103CD0009494155014E1060E236EE80E1B6E030E2D
:103CE0001C6E1D6A1E6A14A423D71750172AEA6A8D
:103CF000400FE96E040EEA22F1C5EFFF19D7020E5C
:103D00000501F45D13E11704EA6A400FE96E040E41
:103D1000EA22EF500101E75D09E1060E236EE80E8D
:103D20001B6E030E1C6E1D6A1E6A02D7010E49D05F
:103D300080A802D0090E236E1B06000E1C5A1D5AC5
:103D40001E5AD8801B54000E1C54000E1D54000E29
:103D50001E5402E3630E236E9492949414A6E8D644
:103D60000401320EC06F030EC16F5F0EC26F06DD1D
:103D7000DFD61750000820E2080E0501F5151CE0FB
:103D8000620E256E450E266E276A25C0E6FFE66E9A
:103D900027C0E6FFC20EE66E010EE66E82EC24F04E
:103DA000286E050EE15E2850C20EE66E010EE66E2C
:103DB000FDEC23F0E552E552010EDF6E94929494EF
:103DC000630E236EB5D61750000826E2080E0501D3
:103DD000F51522E0DFCFE6FFE66A1750E66EE66AE9
:103DE0004D0E256E450E266E276A25C0E6FFE66E4F
:103DF00027C0E6FFC20EE66E010EE66E82EC24F0EE
:103E0000286E090EE15E2850C20EE66E010EE66EC7
:103E1000FDEC23F0E552E552DF5003E0F368F46A6D
:103E200007D01750256E266A17C0F3FF26C0F4FF8F
:103E3000E552E552E7CFD9FF120092928092A00E90
:103E40001B6E860E1C6E010E1D6E1E6A1B501C1012
:103E50001D101E1006E01B06000E1C5A1D5A1E5A8D
:103E6000F5D792828082A00E1B6E860E1C6E010E0C
:103E70001D6E1E6A1B501C101D101E1006E01B0636
:103E8000000E1C5A1D5A1E5AF5D71200D9CFE6FF54
:103E9000E1CFD9FFFE0EDB0403E1929A809A02D0B3
:0C3EA000928A808AE552E7CFD9FF120019
:043EAC00040130518C
:103EB0001F0B010801E012003051600BE842E8429C
:103EC000E842E842E842010801E01200345103E010
:103ED000340501E012003151220A31E0030A24E0E6
:103EE000010A15E0210A0DE0010A01E012000201B9
:103EF000F30E886F000E896F080E8B6F8C6B8A81B2
:103F000021D00201F30E886F000E896F1BD036C4DA
:103F100090F237C491F20201800E8D6F050E8E6F04
:103F2000926B936B8F8F12000201800E886F050ECB
:103F3000896F070E8B6F8C6BC10E8A6F120032C4B3
:103F4000EEF002018A8F12000501806B4B0E816F2B
:103F5000826B836B846B856B080E866F0001E26B4E
:103F60001A0EE66E010EE66EBAEC13F0E552E5525B
:103F70001E0EE66E020EE66EBAEC13F0E552E55246
:103F8000400EE66E400EE66E050EE66EE66A020E26
:103F9000E66EF1EC13F0256E050EE15E2550F3CFD1
:103FA000EAF0F4CFEBF00001EC6BED6BE36B120089
:103FB000D9CFE6FFE1CFD9FFFD0EDBCF06F0FE0E35
:103FC000DBCF07F0050E061801E1075002E0000EF6
:103FD00030D0FB0EDBCF25F0FC0EDBCF26F000014E
:103FE000EA51251816E1EB51261813E1400EE66E52
:103FF000400EE66E050EE66EE66A020EE66EF1EC27
:1040000013F0256E050EE15E2550F3CFEAF0F4CFF4
:10401000EBF0FB0EDBCF25F0FC0EDBCF26F0000132
:10402000EC51251805E1ED51261802E1E36BE86B30
:10403000010EE552E7CFD9FF1200D9CFE6FFE1CF5D
:10404000D9FF0001E26BEA51EB1102E1000E08D04A
:10405000EAC0E9FFEBC0EAFFEF50800B01E0010E80
:10406000000945E1FC0EDBCF25F0EAC0E9FFEBC01B
:10407000EAFFEE52EF50D880255408E2EAC0E9FF8B
:10408000EBC0EAFFEE52FC0EEFCFDBFFE26BFC0E63
:10409000DB50E25D19E2E251EA6A400FE96E050E7B
:1040A000EA22EF50E66EE251E76EFD0EDBCFE9FF4C
:1040B000FE0EDBCFEAFFE750E926000EEA22E552CA
:1040C000E750EF6EE22BE3D7400EE66E400EE66E51
:1040D000050EE66EE66A020EE66EF1EC13F0256E52
:1040E000050EE15E2550F3CFEAF0F4CFEBF00001CE
:1040F000E251E552E7CFD9FF1200D9CFE6FFE1CF79
:10410000D9FF0001E3510CE1FD0EDBCFE4F0FE0E20
:10411000DBCFE5F0FC0EDBCFE8F0010EE96FE36FDB
:10412000E552E7CFD9FF1200D9CFE6FFE1CFD9FFA3
:10413000030EE1260001E3512DE1DF6AFD0EDBCF26
:1041400006F0FE0EDBCF07F0DE5206C0DEFF07C032
:10415000DDFFDD52DF2ADF50256E266AFF0E2518AF
:1041600002E126500BE0010EDBCFE9FFDB2A020E55
:10417000DBCFEAFF01E3DB2AEF50ECE1FD0EDBCF02
:10418000E4F0FE0EDBCFE5F0DF040001E86F010E86
:10419000E96FE36F030EE15C02E2E16AE552E16E72
:1041A000E552E7CFD9FF1200D9CFE6FFE1CFD9FF23
:1041B000030EE1260001E3512EE1DF6AFD0EDBCFA5
:1041C00006F0FE0EDBCF07F0DE5206C0DEFF07C0B2
:1041D000DDFFDD52DF2ADF50256E266AFF0E25182F
:1041E00002E126500CE0010EDBCFF6FFDB2A020EC7
:1041F000DBCFF7FF01E3DB2A0800F550EBE1FD0E12
:10420000DBCFE4F0FE0EDBCFE5F0DFCFE8F000011E
:10421000E96B010EE36F030EE15C02E2E16AE55235
:10422000E16EE552E7CFD9FF1200D9CFE6FFE1CF2B
:10423000D9FF020EE1260001EC51ED1102E1000E62
:1042400008D0ECC0E9FFEDC0EAFFEF50800B01E0C1
:10425000010E000901E084D0030EE35D01E1E36B90
:10426000E35101E17DD0020EE35D16E1E66A000E46
:10427000E66EE66A010EE66E020EE66EF1EC13F0F3
:10428000256E050EE15E2550F3CFECF0F4CFEDF096
:104290000001030EE36F64D0E30562E1400E256E7A
:1042A000266AE851255C000E265803E2400EDF6EB8
:1042B00002D0E8C0DFFFDF50E85DE86F000EE66F78
:1042C000050EE76F010EDFCFDBFFE95116E1010EAE
:1042D000DB5028E0E4C0F6FFE5C0F7FF0800F5502A
:1042E000E6C0E9FFE7C0EAFFEF6EE62B000EE7232A
:1042F000E42BE523010EDB06EAD7010EDB5012E0CA
:10430000E4C0E9FFE5C0EAFFEF50E6C0E9FFE7C01F
:10431000EAFFEF6EE62B000EE723E42BE523010E08
:10432000DB06EBD70001E85107E1400EDF5C02E15C
:10433000020E01D0030EE36FDFCFE6FF000EE66E44
:10434000050EE66E010EE66E020EE66EF1EC13F05F
:10435000256E050EE15E2550F3CFECF0F4CFEDF0C5
:10436000020EE15C02E2E16AE552E16EE552E7CF5E
:04437000D9FF12005F
:0C437400D9CFE6FFE1CFD9FF060EE1260D
:10438000200E0201E76E7219E8AE02D0E73402D0C7
:10439000E750725D01E2B8D06D50020B01E0B4D07D
:1043A0000001E35169E1400EE66EE66AE66A400EFE
:1043B000E66E010EE66E48EC23F0256E050EE15E1A
:1043C0002550400EE66E400EE66E010EE66E1DECC8
:1043D00020F0E552E552E552DE6EDD6AD9CFE9FF05
:1043E000DACFEAFFEE50ED1047E0000EE66E020E67
:1043F000E66EDECFE6FFDDCFE6FF800EE66E010E55
:10440000E66EDECFE6FFDDCFE6FF400EE66E010E84
:10441000E66E0FEC08F0256E0A0EE15E2550020EE6
:10442000F3CFDBFF030EF4CFDBFF0501F5A124D0B2
:10443000400E256E450E266E276A25C0E6FFE66E05
:1044400027C0E6FFC20EE66E010EE66E82EC24F097
:10445000286E050EE15E2850C20EE66E010EE66E75
:10446000FDEC23F0E552E552400EE66E010EE66EDD
:10447000FDEC23F0E552E55215EC21F015EC21F0AE
:104480000001E3513FE1010E185C3CE2176A72EC57
:104490001DF01750000836E20001E35133E11750D8
:1044A000E66E400EE66E040EE66E7DEC20F0E55200
:1044B000E552E552176A0501F5A324D0320E256EA8
:1044C000450E266E276A25C0E6FFE66E27C0E6FF8A
:1044D000C20EE66E010EE66E82EC24F0286E050E2A
:1044E000E15E2850C20EE66E010EE66EFDEC23F092
:1044F000E552E552400EE66E040EE66EFDEC23F04A
:10450000E552E55215EC21F0060EE15C02E2E16AAB
:0C451000E552E16EE552E7CFD9FF120042
:04451C000D0A5374BD
:10452000617274696E670D0A002553202558202595
:1045300058000D0A46726F6D20475049423A2000DC
:104540000D0A46726F6D205553423A20000D0A52F3
:10455000583A2025642074696D656F757420256450
:1045600020002074696D656F757420003C25303221
:10457000583E2553002563000D0A003C4552523E2B
:10458000003C454F493E002553003C253032583E03
:104590000044415441206C656E0025533A25642047
:1045A00000434D44206C656E3A20256420000D0ABE
:1045B00054583A2025582025582000536570203043
:1045C000362032303135005072656C6F6769782063
:1045D000475049422D55534220436F6E74726F6CA1
:1045E0006C65722076657273696F6E20362E32208C
:1045F00025530D0A004E6565642068656C703F2088
:104600004C6F6F6B20696E2074686520736F7572D4
:10461000636520636F6465210D0A00256400656E83
:104620006400646562756700766572007472670085
:104630007372710073706F6C6C0073617665636682
:104640006700727374007265616400726561645F13
:10465000746D6F5F6D73006D6F6465006C6F6E00DD
:104660006C6F63006966630068656C7000656F74E9
:1046700000656F745F6368617200656F7300656FDA
:104680006900636C72006175746F0061646472002C
:10469000FE0EE3CFE9FFFF0EE3CFEAFFE9CFF3FF22
:1046A000EACFF4FFFB0EE35003E1FC0EE35009E018
:1046B000FB0EE30602E2FC0EE306FD0EE350EE6E97
:1046C000F1D71200FF0EE3CFF8FFE552FF0EE3CF64
:1046D000F7FFE552FF0EE3CFF6FFE552E66AE66A22
:1046E000E66A0900F55209E0FD0EE32A05E1FE0E37
:1046F000E32A02E1FF0EE32AF4D7FD0EE3CF05F033
:10470000FE0EE3CF06F0FF0EE3CF07F01200FD0E22
:10471000E3CFF6FFFE0EE3CFF7FFFF0EE3CFF8FF88
:10472000FB0EE3CFE9FFFC0EE3CFEAFFF90EE35007
:1047300003E1FA0EE3500BE0F90EE30602E2FA0E93
:10474000E306EE500900F55C02E1F566EFD71200D2
:10475000FE0EE3CFE9FFFF0EE3CFEAFFF36AF46A50
:0C476000EE5203E0F34AF42AFBD71200EB
:04476C000C0EAF6E12
:10477000B06AB896AC98AB8EAB88AB9A9D989D9A70
:10478000D08E9F8AF28EAC90AB9CAC9AAC8AAC94E3
:104790000001E191E06B1200D9CFE6FFE1CFD9FF34
:1047A0009EB803D014D80400FBD7FE0EDB50AD6ECC
:1047B000E552E7CFD9FF12009EBA03D0040007D814
:1047C000FBD7AE5000D012009EBA010C000CD9CF1E
:1047D000E6FFE1CFD9FFE652ABA204D0AC9AAC8A97
:1047E000AB98AB88ABA404D0AE50DF6EAC9AAC8A69
:1047F000E552E552E7CFD9FF1200D9CFE6FFE1CF6E
:10480000D9FFFD0EDBCFE9FFFE0EDBCFEAFFEF5055
:1048100010E0FD0EDBCFE9FFFE0EDBCFEAFFEF502D
:10482000E66EBADFE552FD0EDB2AFE0EEAE3DB2A76
:0A483000E8D7E552E7CFD9FF1200E8
:06483A0012010002020061
:104840000008D8040A000001010200010902430027
:10485000020100C032090400000102020100052427
:1048600000100104240202052406000105240100B1
:10487000010705810308000209040100020A000083
:104880000007050202400000070582024000000404
:1048900003090434034D006900630072006F006374
:1048A0000068006900700020005400650063006823
:1048B000006E006F006C006F0067007900200049F7
:1048C000006E0063002E00340343004400430020C8
:1048D00000520053002D003200330032002000450A
:1048E000006D0075006C006100740069006F006E5F
:1048F000002000440065006D006F004C488F489315
:0349000048C7485D
:0C490400D9CFE6FFDACFE6FFE1CFD9FF04
:10491000E2CFDAFFE652E652E652E652D950F90FFC
:10492000256EFF0EDA20266E020E25C0DBFF030E79
:1049300026C0DBFF020EDBCFE6FF030EDBCFE6FF78
:10494000F90EDBCFE6FFFA0EDBCFE6FFFB0EDBCF87
:10495000E6FFD950FC0FE66EFF0EDA20E66E32EC71
:1049600000F0256E070EE15C02E2E16AE552E16EBD
:104970002550F3CFDEFFF4CFDDFFFC0EDBCFE9FFE8
:10498000FD0EDBCFEAFFEF6ADECF25F0DDCF26F0AC
:1049900025C0F3FF26C0F4FF040EE15C02E2E16AE9
:1049A000E552E16EE552E5CFDAFFE7CFD9FF12001D
:1049B0001E0EF66E000EF76E000EF86E0101090075
:1049C000F550F46F0900F550F56F03E1F46701D07D
:1049D0003DD00900F550EF6F0900F550F06F090068
:1049E000F550F16F09000900F550E96E0900F55026
:1049F000EA6E090009000900F550F26F0900F55050
:104A0000F36F09000900F6CFF6F1F7CFF7F1F8CF11
:104A1000F8F1EFC1F6FFF0C1F7FFF1C1F8FF0101B6
:104A2000F25302E1F35307E00900F550EE6EF2078E
:104A3000F8E2F307F9D7F6C1F6FFF7C1F7FFF8C1BF
:0E4A4000F8FF0101F407000EF55BBFD712006E
:024A4E00D9CFBE
:104A5000E6FFDACFE6FFE1CFD9FFE2CFDAFFFB0EC8
:104A6000DBCF25F0FC0EDBCF26F00001800E2614F4
:104A70001AE1FB0EDBCFE9FFFC0EDBCFEAFFEECF46
:104A8000F3FFEDCFF4FFEE2A000EEF22F3CFE9FFA4
:104A9000F4CFEAFFFD0EDBCFEFFFEF50266AF36E97
:104AA00026C0F4FF10D0FB0EDB50FE0806E1FD0E21
:104AB000DBCFE6FF0DEC26F005D0FD0EDBCFE6FFE9
:104AC00003EC00F0E552E552E5CFDAFFE7CFD9FF7E
:024AD0001200D2
:0E4AD20004500B02F3CF00F0F4CF01F00C0201
:104AE000F3500126000EF420026E04500D02F35024
:104AF0000226000EF420036E04500E02F35003262B
:104B000005500B02F3500126F4500222000E03223E
:104B100005500C02F3500226F450032205500D02FA
:104B2000F350032606500B02F3500226F4500322E2
:104B300006500C02F350032607500B02F3500326D5
:024B4000120061
:0E4B4200F36AF46AFF0EE124E96EFF0EE22032
:104B5000EA6EED660DD0400EEF640AD05A0EEF6497
:104B600006D0600EEF6404D07B0EEF6001D0F32A14
:104B70001200F36AF46AFF0EE124E96EFF0EE220F0
:104B8000EA6EED6607D02F0EEF6404D03A0EEF60A8
:064B900001D0F32A12001F
:0A4B9600036A026A016A006A200E39
:104BA000E76ED890043605360636073600360136ED
:104BB000023603360B50005C0C5001580D50025861
:104BC0000E50035809E30B50005E0C50015A0D5073
:0E4BD000025A0E50035A042AE72EE4D71200B0
:024BDE00000EC7
:104BE000F36E00EE00F0080E01D81200EA6002D069
:0E4BF000EE6AFCD7F350E9601200EE6AFCD7C3
:024BFE0013EEB4
:104C000000F023EE00F0F86A0A9CD8EC24F0FFECE8
:0A4C100007F045EC06F0FBD7120098
:064C1A00FF0EE350ACBAEE
:104C200004D0AF6AAB8EAC8A949CACA2FED7AD6EBA
:064C3000F36EF46A1200AD
:0A4C3600FF0EE3502D6E1B0E00D0A0
:104C400001D0200EE76EE72EFED72D2EFAD700D02A
:024C5000120050
:0E4C5200FF0EE350E84E1200000000D000D02C
:084C600000D0E82EFAD7120083
:084C68003031323334353637A8
:094C700038396162636465660075
:074C79008B4656198646E048
:104C8000198246701B7E46BA1B7A46961C7146FCFA
:104C90001D6D46201D6846BC1A6446FE1A60468695
:104CA0001E5C46B21E57468E1F4B463A214646743E
:104CB000204246C8213A46B02434463022304624A9
:104CC000232C468C232846261B224626241E4600DB
:064CD000004E554C4C00A3
:020000040030CA
:0100000024DB
:010001000EF0
:010002003FBE
:010003001EDE
:010005008179
:010006008178
:010008000FE8
:01000900C036
:01000A000FE6
:01000B00E014
:01000C000FE4
:01000D0040B2
:00000001FF
